###############################################################################
#                                                                             #
# IAR ELF Linker V5.41.0.51741/W32 for ARM              10/Jan/2014  09:52:10 #
# Copyright (C) 2007-2009 IAR Systems AB.                                     #
#                                                                             #
#    Output file  =  E:\WIZnet 产品文档\W5500\W5500\Application               #
#                    Reference\DHCP test\DHCP test\Debug\Exe\app.out          #
#    Map file     =  E:\WIZnet 产品文档\W5500\W5500\Application               #
#                    Reference\DHCP test\DHCP test\Debug\List\app.map         #
#    Command line =  "E:\WIZnet 产品文档\W5500\W5500\Application              #
#                    Reference\DHCP test\DHCP test\Debug\Obj\SPI2.o"          #
#                    "E:\WIZnet 产品文档\W5500\W5500\Application              #
#                    Reference\DHCP test\DHCP test\Debug\Obj\at24c16.o"       #
#                    "E:\WIZnet 产品文档\W5500\W5500\Application              #
#                    Reference\DHCP test\DHCP test\Debug\Obj\core_cm3.o"      #
#                    "E:\WIZnet 产品文档\W5500\W5500\Application              #
#                    Reference\DHCP test\DHCP test\Debug\Obj\device.o"        #
#                    "E:\WIZnet 产品文档\W5500\W5500\Application              #
#                    Reference\DHCP test\DHCP test\Debug\Obj\dhcp.o"          #
#                    "E:\WIZnet 产品文档\W5500\W5500\Application              #
#                    Reference\DHCP test\DHCP test\Debug\Obj\main.o"          #
#                    "E:\WIZnet 产品文档\W5500\W5500\Application              #
#                    Reference\DHCP test\DHCP test\Debug\Obj\mcu_init.o"      #
#                    "E:\WIZnet 产品文档\W5500\W5500\Application              #
#                    Reference\DHCP test\DHCP test\Debug\Obj\md5.o"           #
#                    "E:\WIZnet 产品文档\W5500\W5500\Application              #
#                    Reference\DHCP test\DHCP test\Debug\Obj\misc.o"          #
#                    "E:\WIZnet 产品文档\W5500\W5500\Application              #
#                    Reference\DHCP test\DHCP test\Debug\Obj\socket.o"        #
#                    "E:\WIZnet 产品文档\W5500\W5500\Application              #
#                    Reference\DHCP test\DHCP test\Debug\Obj\sockutil.o"      #
#                    "E:\WIZnet 产品文档\W5500\W5500\Application              #
#                    Reference\DHCP test\DHCP test\Debug\Obj\startup_stm32f10 #
#                    x_hd.o" "E:\WIZnet 产品文档\W5500\W5500\Application      #
#                    Reference\DHCP test\DHCP test\Debug\Obj\stm32f10x_bkp.o" #
#                     "E:\WIZnet 产品文档\W5500\W5500\Application             #
#                    Reference\DHCP test\DHCP test\Debug\Obj\stm32f10x_flash. #
#                    o" "E:\WIZnet 产品文档\W5500\W5500\Application           #
#                    Reference\DHCP test\DHCP test\Debug\Obj\stm32f10x_gpio.o #
#                    " "E:\WIZnet 产品文档\W5500\W5500\Application            #
#                    Reference\DHCP test\DHCP test\Debug\Obj\stm32f10x_it.o"  #
#                    "E:\WIZnet 产品文档\W5500\W5500\Application              #
#                    Reference\DHCP test\DHCP test\Debug\Obj\stm32f10x_rcc.o" #
#                     "E:\WIZnet 产品文档\W5500\W5500\Application             #
#                    Reference\DHCP test\DHCP test\Debug\Obj\stm32f10x_spi.o" #
#                     "E:\WIZnet 产品文档\W5500\W5500\Application             #
#                    Reference\DHCP test\DHCP test\Debug\Obj\stm32f10x_usart. #
#                    o" "E:\WIZnet 产品文档\W5500\W5500\Application           #
#                    Reference\DHCP test\DHCP test\Debug\Obj\system_stm32f10x #
#                    .o" "E:\WIZnet 产品文档\W5500\W5500\Application          #
#                    Reference\DHCP test\DHCP test\Debug\Obj\util.o"          #
#                    "E:\WIZnet 产品文档\W5500\W5500\Application              #
#                    Reference\DHCP test\DHCP test\Debug\Obj\w5500.o" -o      #
#                    "E:\WIZnet 产品文档\W5500\W5500\Application              #
#                    Reference\DHCP test\DHCP test\Debug\Exe\app.out" --map   #
#                    "E:\WIZnet 产品文档\W5500\W5500\Application              #
#                    Reference\DHCP test\DHCP test\Debug\List\app.map"        #
#                    --config "E:\WIZnet 产品文档\W5500\W5500\Application     #
#                    Reference\DHCP test\DHCP test\app.icf" --semihosting     #
#                    --entry __iar_program_start                              #
#                                                                             #
#                                                                             #
###############################################################################

*******************************************************************************
*** RUNTIME MODEL ATTRIBUTES
***

__endian      = little
__thumb_aware = enabled


*******************************************************************************
*** PLACEMENT SUMMARY
***

"A1":  place at 0x08000000 { ro section .intvec };
"P1":  place in [from 0x08000000 to 0x0803ffff] { ro };
"P2":  place in [from 0x20000000 to 0x2000bfff] {
          rw, block CSTACK, block HEAP };

  Section            Kind        Address    Size  Object
  -------            ----        -------    ----  ------
"A1":                                      0x130
  .intvec            ro code  0x08000000   0x130  startup_stm32f10x_hd.o [1]
                            - 0x08000130   0x130

"P1":                                     0x4e6c
  .text              ro code  0x08000130  0x1460  dhcp.o [1]
  .text              ro code  0x08001590   0xcc2  xprintffull.o [3]
  .text              ro code  0x08002254   0x4a0  socket.o [1]
  .text              ro code  0x080026f4   0x420  w5500.o [1]
  .text              ro code  0x08002b14   0x340  stm32f10x_rcc.o [1]
  .text              ro code  0x08002e54   0x246  DblDiv.o [4]
  .text              ro code  0x0800309c   0x1f4  mcu_init.o [1]
  .text              ro code  0x08003290   0x1a2  DblMul.o [4]
  .text              ro code  0x08003434   0x18a  stm32f10x_usart.o [1]
  .text              ro code  0x080035c0   0x17e  DblSub.o [4]
  .text              ro code  0x08003740   0x15c  stm32f10x_gpio.o [1]
  .text              ro code  0x0800389c   0x158  system_stm32f10x.o [1]
  .text              ro code  0x080039f4   0x130  device.o [1]
  .text              ro code  0x08003b24   0x12e  I64DivMod.o [4]
  .text              ro code  0x08003c54   0x108  xdscale.o [3]
  .text              ro code  0x08003d5c   0x104  util.o [1]
  .text              ro code  0x08003e60    0xe6  DblAdd.o [4]
  .text              ro code  0x08003f46    0xc6  xdnorm.o [3]
  .text              ro code  0x0800400c    0xb4  SPI2.o [1]
  .text              ro code  0x080040c0    0xa0  misc.o [1]
  .text              ro code  0x08004160    0x7c  stm32f10x_spi.o [1]
  .text              ro code  0x080041dc    0x70  ABImemcpy.o [4]
  .text              ro code  0x0800424c    0x6c  main.o [1]
  .text              ro code  0x080042b8    0x66  ABImemset.o [4]
  .text              ro code  0x08004320    0x62  memcmp.o [4]
  .text              ro code  0x08004384    0x58  memchr.o [4]
  .text              ro code  0x080043dc    0x56  DblToI32.o [4]
  .text              ro code  0x08004434    0x44  strcpy.o [4]
  .rodata            const    0x08004478    0x40  dhcp.o [1]
  .text              ro code  0x080044b8    0x3c  at24c16.o [1]
  .text              ro code  0x080044f4    0x3c  stm32f10x_flash.o [1]
  .text              ro code  0x08004530    0x36  strlen.o [4]
  .rodata            const    0x08004568    0x34  dhcp.o [1]
  .rodata            const    0x0800459c    0x30  dhcp.o [1]
  .text              ro code  0x080045cc    0x30  sprintf.o [3]
  .text              ro code  0x080045fc    0x2e  DblCmpLe.o [4]
  .text              ro code  0x0800462c    0x2e  DblCmpGe.o [4]
  .text              ro code  0x0800465c    0x2e  I32ToDbl.o [4]
  .rodata            const    0x0800468c    0x2c  dhcp.o [1]
  .rodata            const    0x080046b8    0x2c  dhcp.o [1]
  .rodata            const    0x080046e4    0x2c  dhcp.o [1]
  .rodata            const    0x08004710    0x28  dhcp.o [1]
  .rodata            const    0x08004738    0x28  dhcp.o [1]
  .rodata            const    0x08004760    0x28  dhcp.o [1]
  .text              ro code  0x08004788    0x26  sockutil.o [1]
  .rodata            const    0x080047b0    0x24  dhcp.o [1]
  .rodata            const    0x080047d4    0x24  dhcp.o [1]
  .rodata            const    0x080047f8    0x24  dhcp.o [1]
  .rodata            const    0x0800481c    0x24  dhcp.o [1]
  .rodata            const    0x08004840    0x24  dhcp.o [1]
  .rodata            const    0x08004864    0x24  dhcp.o [1]
  .rodata            const    0x08004888    0x24  main.o [1]
  .text              ro code  0x080048ac    0x24  copy_init2.o [4]
  .iar.init_table    const    0x080048d0    0x24  - Linker created -
  .rodata            const    0x080048f4    0x20  dhcp.o [1]
  .rodata            const    0x08004914    0x20  dhcp.o [1]
  .rodata            const    0x08004934    0x20  dhcp.o [1]
  .rodata            const    0x08004954    0x20  dhcp.o [1]
  .rodata            const    0x08004974    0x20  dhcp.o [1]
  .rodata            const    0x08004994    0x20  dhcp.o [1]
  .rodata            const    0x080049b4    0x20  w5500.o [1]
  .text              ro code  0x080049d4    0x20  printf.o [3]
  .text              ro code  0x080049f4    0x20  data_init2.o [4]
  .rodata            const    0x08004a14    0x1c  dhcp.o [1]
  .rodata            const    0x08004a30    0x1c  dhcp.o [1]
  .rodata            const    0x08004a4c    0x1c  dhcp.o [1]
  .rodata            const    0x08004a68    0x1c  dhcp.o [1]
  .rodata            const    0x08004a84    0x1c  dhcp.o [1]
  .rodata            const    0x08004aa0    0x1c  dhcp.o [1]
  .text              ro code  0x08004abc    0x1c  iarwstd.o [5]
  .text              ro code  0x08004ad8    0x1a  stm32f10x_it.o [1]
  .text              ro code  0x08004af2    0x1a  zero_init2.o [4]
  .rodata            const    0x08004b0c    0x18  dhcp.o [1]
  .rodata            const    0x08004b24    0x18  dhcp.o [1]
  .rodata            const    0x08004b3c    0x18  dhcp.o [1]
  .rodata            const    0x08004b54    0x18  dhcp.o [1]
  .rodata            const    0x08004b6c    0x18  dhcp.o [1]
  .rodata            const    0x08004b84    0x18  dhcp.o [1]
  .rodata            const    0x08004b9c    0x18  dhcp.o [1]
  .rodata            const    0x08004bb4    0x18  dhcp.o [1]
  .rodata            const    0x08004bcc    0x18  dhcp.o [1]
  .rodata            const    0x08004be4    0x18  main.o [1]
  .rodata            const    0x08004bfc    0x18  socket.o [1]
  .rodata            const    0x08004c14    0x18  w5500.o [1]
  .text              ro code  0x08004c2c    0x18  cmain.o [4]
  .text              ro code  0x08004c44    0x16  strchr.o [4]
  .text              ro code  0x08004c5a    0x16  device.o [1]
  .text              ro code  0x08004c70    0x16  dhcp.o [1]
  .text              ro code  0x08004c86    0x16  xprout.o [3]
  .rodata            const    0x08004c9c    0x14  dhcp.o [1]
  .rodata            const    0x08004cb0    0x14  dhcp.o [1]
  .rodata            const    0x08004cc4    0x14  dhcp.o [1]
  .rodata            const    0x08004cd8    0x14  dhcp.o [1]
  .rodata            const    0x08004cec    0x14  dhcp.o [1]
  .rodata            const    0x08004d00    0x14  dhcp.o [1]
  .rodata            const    0x08004d14    0x14  dhcp.o [1]
  .rodata            const    0x08004d28    0x14  dhcp.o [1]
  .rodata            const    0x08004d3c    0x14  dhcp.o [1]
  .rodata            const    0x08004d50    0x14  dhcp.o [1]
  .text              ro code  0x08004d64    0x14  exit.o [5]
  .rodata            const    0x08004d78    0x10  dhcp.o [1]
  .rodata            const    0x08004d88    0x10  dhcp.o [1]
  .rodata            const    0x08004d98    0x10  dhcp.o [1]
  .rodata            const    0x08004da8    0x10  dhcp.o [1]
  .rodata            const    0x08004db8    0x10  dhcp.o [1]
  .rodata            const    0x08004dc8    0x10  dhcp.o [1]
  .text              ro code  0x08004dd8    0x10  startup_stm32f10x_hd.o [1]
  .text              ro code  0x08004de8     0xe  div.o [3]
  .text              ro code  0x08004df8     0xa  cexit.o [4]
  .text              ro code  0x08004e02     0xa  xsprout.o [3]
  .rodata            const    0x08004e0c     0x8  device.o [1]
  .rodata            const    0x08004e14     0x8  dhcp.o [1]
  .rodata            const    0x08004e1c     0x8  dhcp.o [1]
  .rodata            const    0x08004e24     0x8  dhcp.o [1]
  .rodata            const    0x08004e2c     0x8  xprintffull.o [3]
  .text              ro code  0x08004e34     0x6  exit.o [3]
  .rodata            const    0x08004e3c     0x4  device.o [1]
  .rodata            const    0x08004e40     0x4  device.o [1]
  .rodata            const    0x08004e44     0x4  device.o [1]
  .rodata            const    0x08004e48     0x4  device.o [1]
  .rodata            const    0x08004e4c     0x4  dhcp.o [1]
  .text              ro code  0x08004e50     0x2  I64DivZer.o [4]
  .text              ro code  0x08004e52     0x4  startup_stm32f10x_hd.o [1]
  .text              ro code  0x08004e56     0x4  startup_stm32f10x_hd.o [1]
  .text              ro code  0x08004e5a     0x4  startup_stm32f10x_hd.o [1]
  .text              ro code  0x08004e5e     0x4  startup_stm32f10x_hd.o [1]
  .text              ro code  0x08004e62     0x4  startup_stm32f10x_hd.o [1]
  .text              ro code  0x08004e66     0x4  startup_stm32f10x_hd.o [1]
  .text              ro code  0x08004e6a     0x4  startup_stm32f10x_hd.o [1]
  .text              ro code  0x08004e6e     0x4  startup_stm32f10x_hd.o [1]
  .text              ro code  0x08004e72     0x4  startup_stm32f10x_hd.o [1]
  .text              ro code  0x08004e76     0x4  startup_stm32f10x_hd.o [1]
  .text              ro code  0x08004e7a     0x4  startup_stm32f10x_hd.o [1]
  .text              ro code  0x08004e7e     0x4  startup_stm32f10x_hd.o [1]
  .text              ro code  0x08004e82     0x4  startup_stm32f10x_hd.o [1]
  .text              ro code  0x08004e86     0x4  startup_stm32f10x_hd.o [1]
  .text              ro code  0x08004e8a     0x4  startup_stm32f10x_hd.o [1]
  .text              ro code  0x08004e8e     0x4  startup_stm32f10x_hd.o [1]
  .text              ro code  0x08004e92     0x4  startup_stm32f10x_hd.o [1]
  .text              ro code  0x08004e96     0x4  startup_stm32f10x_hd.o [1]
  .text              ro code  0x08004e9a     0x4  startup_stm32f10x_hd.o [1]
  .text              ro code  0x08004e9e     0x4  startup_stm32f10x_hd.o [1]
  .text              ro code  0x08004ea2     0x4  startup_stm32f10x_hd.o [1]
  .text              ro code  0x08004ea6     0x4  startup_stm32f10x_hd.o [1]
  .text              ro code  0x08004eaa     0x4  startup_stm32f10x_hd.o [1]
  .text              ro code  0x08004eae     0x4  startup_stm32f10x_hd.o [1]
  .text              ro code  0x08004eb2     0x4  startup_stm32f10x_hd.o [1]
  .text              ro code  0x08004eb6     0x4  startup_stm32f10x_hd.o [1]
  .text              ro code  0x08004eba     0x4  startup_stm32f10x_hd.o [1]
  .text              ro code  0x08004ebe     0x4  startup_stm32f10x_hd.o [1]
  .text              ro code  0x08004ec2     0x4  startup_stm32f10x_hd.o [1]
  .text              ro code  0x08004ec6     0x4  startup_stm32f10x_hd.o [1]
  .text              ro code  0x08004eca     0x4  startup_stm32f10x_hd.o [1]
  .text              ro code  0x08004ece     0x4  startup_stm32f10x_hd.o [1]
  .text              ro code  0x08004ed2     0x4  startup_stm32f10x_hd.o [1]
  .text              ro code  0x08004ed6     0x4  startup_stm32f10x_hd.o [1]
  .text              ro code  0x08004eda     0x4  startup_stm32f10x_hd.o [1]
  .text              ro code  0x08004ede     0x4  startup_stm32f10x_hd.o [1]
  .text              ro code  0x08004ee2     0x4  startup_stm32f10x_hd.o [1]
  .text              ro code  0x08004ee6     0x4  startup_stm32f10x_hd.o [1]
  .text              ro code  0x08004eea     0x4  startup_stm32f10x_hd.o [1]
  .text              ro code  0x08004eee     0x4  startup_stm32f10x_hd.o [1]
  .text              ro code  0x08004ef2     0x4  startup_stm32f10x_hd.o [1]
  .text              ro code  0x08004ef6     0x4  startup_stm32f10x_hd.o [1]
  .text              ro code  0x08004efa     0x4  startup_stm32f10x_hd.o [1]
  .text              ro code  0x08004efe     0x4  startup_stm32f10x_hd.o [1]
  .text              ro code  0x08004f02     0x4  startup_stm32f10x_hd.o [1]
  .text              ro code  0x08004f06     0x4  startup_stm32f10x_hd.o [1]
  .text              ro code  0x08004f0a     0x4  startup_stm32f10x_hd.o [1]
  .text              ro code  0x08004f0e     0x4  startup_stm32f10x_hd.o [1]
  .text              ro code  0x08004f12     0x4  startup_stm32f10x_hd.o [1]
  .text              ro code  0x08004f16     0x4  startup_stm32f10x_hd.o [1]
  .text              ro code  0x08004f1a     0x4  startup_stm32f10x_hd.o [1]
  .text              ro code  0x08004f1e     0x4  startup_stm32f10x_hd.o [1]
  .text              ro code  0x08004f22     0x4  startup_stm32f10x_hd.o [1]
  .text              ro code  0x08004f26     0x4  startup_stm32f10x_hd.o [1]
  .text              ro code  0x08004f2a     0x4  startup_stm32f10x_hd.o [1]
  .text              ro code  0x08004f2e     0x4  startup_stm32f10x_hd.o [1]
  .text              ro code  0x08004f32     0x4  startup_stm32f10x_hd.o [1]
  .text              ro code  0x08004f36     0x4  startup_stm32f10x_hd.o [1]
  .text              ro code  0x08004f3a     0x4  startup_stm32f10x_hd.o [1]
  .text              ro code  0x08004f3e     0x4  startup_stm32f10x_hd.o [1]
  .text              ro code  0x08004f42     0x4  startup_stm32f10x_hd.o [1]
  .text              ro code  0x08004f46     0x4  startup_stm32f10x_hd.o [1]
  .text              ro code  0x08004f4a     0x4  startup_stm32f10x_hd.o [1]
  .text              ro code  0x08004f4e     0x4  startup_stm32f10x_hd.o [1]
  .text              ro code  0x08004f52     0x4  startup_stm32f10x_hd.o [1]
  .text              ro code  0x08004f56     0x4  startup_stm32f10x_hd.o [1]
  .text              ro code  0x08004f5a     0x4  startup_stm32f10x_hd.o [1]
  .text              ro code  0x08004f5e     0x4  startup_stm32f10x_hd.o [1]
  .text              ro code  0x08004f62     0x4  startup_stm32f10x_hd.o [1]
  .text              ro code  0x08004f66     0x4  low_level_init.o [3]
  Initializer bytes  ro data  0x08004f6c    0x30  <for P2 s0>
                            - 0x08004f9c  0x4e6c

"P2", part 1 of 3:                         0x400
  CSTACK                      0x20000000   0x400  <Block>
    CSTACK           uninit   0x20000000   0x400  <Block tail>
                            - 0x20000400   0x400

"P2", part 2 of 3:                          0x30
  P2 s0                       0x20000400    0x30  <Init block>
    .data            inited   0x20000400    0x10  stm32f10x_rcc.o [1]
    .data            inited   0x20000410     0x4  dhcp.o [1]
    .data            inited   0x20000414     0x4  dhcp.o [1]
    .data            inited   0x20000418     0x4  dhcp.o [1]
    .data            inited   0x2000041c     0x4  dhcp.o [1]
    .data            inited   0x20000420     0x4  dhcp.o [1]
    .data            inited   0x20000424     0x4  dhcp.o [1]
    .data            inited   0x20000428     0x4  dhcp.o [1]
    .data            inited   0x2000042c     0x4  stm32f10x_rcc.o [1]
                            - 0x20000430    0x30

"P2", part 3 of 3:                         0x470
  .bss               zero     0x20000430   0x400  dhcp.o [1]
  .bss               zero     0x20000830    0x24  device.o [1]
  .bss               zero     0x20000854    0x10  w5500.o [1]
  .bss               zero     0x20000864    0x10  w5500.o [1]
  .bss               zero     0x20000874     0x4  dhcp.o [1]
  .bss               zero     0x20000878     0x4  dhcp.o [1]
  .bss               zero     0x2000087c     0x4  dhcp.o [1]
  .bss               zero     0x20000880     0x4  dhcp.o [1]
  .bss               zero     0x20000884     0x4  dhcp.o [1]
  .bss               zero     0x20000888     0x4  dhcp.o [1]
  .bss               zero     0x2000088c     0x4  dhcp.o [1]
  .bss               zero     0x20000890     0x4  iarwstd.o [5]
  .bss               zero     0x20000894     0x2  socket.o [1]
  .bss               zero     0x20000896     0x2  util.o [1]
  .bss               zero     0x20000898     0x1  dhcp.o [1]
  .bss               zero     0x20000899     0x1  dhcp.o [1]
  .bss               zero     0x2000089a     0x1  dhcp.o [1]
  .bss               zero     0x2000089b     0x1  dhcp.o [1]
  .bss               zero     0x2000089c     0x1  util.o [1]
                            - 0x2000089d   0x46d


*******************************************************************************
*** INIT TABLE
***

          Address     Size
          -------     ----
Zero (__iar_zero_init2)
    1 destination range, total size 0x46d:
          0x20000430  0x46d

Copy (__iar_copy_init2)
    1 source range, total size 0x30 (100% of destination):
          0x08004f6c   0x30
    1 destination range, total size 0x30:
          0x20000400   0x30


*******************************************************************************
*** MODULE SUMMARY
***

    Module                  ro code  ro data  rw data
    ------                  -------  -------  -------
E:\WIZnet 产品文档\W5500\W5500\Application Reference\DHCP test\DHCP test\Debug\Obj: [1]
    SPI2.o                      180
    at24c16.o                    60
    device.o                    326       24       36
    dhcp.o                    5 238    1 560    1 084
    main.o                      108       60
    mcu_init.o                  500
    misc.o                      160
    socket.o                  1 184       24        2
    sockutil.o                   38
    startup_stm32f10x_hd.o      596
    stm32f10x_flash.o            60
    stm32f10x_gpio.o            348
    stm32f10x_it.o               26
    stm32f10x_rcc.o             832       20       20
    stm32f10x_spi.o             124
    stm32f10x_usart.o           394
    system_stm32f10x.o          344
    util.o                      260                 3
    w5500.o                   1 056       56       32
    -------------------------------------------------
    Total:                   11 834    1 744    1 177

command line: [2]
    -------------------------------------------------
    Total:

dl7M_tl_in.a: [3]
    div.o                        14
    exit.o                        6
    low_level_init.o              4
    printf.o                     32
    sprintf.o                    48
    xdnorm.o                    198
    xdscale.o                   264
    xprintffull.o             3 266        8
    xprout.o                     22
    xsprout.o                    10
    -------------------------------------------------
    Total:                    3 864        8

rt7M_tl.a: [4]
    ABImemcpy.o                 112
    ABImemset.o                 102
    DblAdd.o                    230
    DblCmpGe.o                   46
    DblCmpLe.o                   46
    DblDiv.o                    582
    DblMul.o                    418
    DblSub.o                    382
    DblToI32.o                   86
    I32ToDbl.o                   46
    I64DivMod.o                 302
    I64DivZer.o                   2
    cexit.o                      10
    cmain.o                      24
    copy_init2.o                 36
    data_init2.o                 32
    memchr.o                     88
    memcmp.o                     98
    strchr.o                     22
    strcpy.o                     68
    strlen.o                     54
    zero_init2.o                 26
    -------------------------------------------------
    Total:                    2 812

shb_l.a: [5]
    exit.o                       20
    iarwstd.o                    28                 4
    -------------------------------------------------
    Total:                       48                 4

    Gaps                         24        8
    Linker created                        38    1 024
-----------------------------------------------------
    Grand Total:             18 582    1 798    2 205


*******************************************************************************
*** ENTRY LIST
***

Entry                      Address   Size  Type      Object
-----                      -------   ----  ----      ------
ADC1_2_IRQHandler       0x08004ebf         Code  Wk  startup_stm32f10x_hd.o [1]
ADC3_IRQHandler         0x08004f33         Code  Wk  startup_stm32f10x_hd.o [1]
ADCPrescTable           0x2000042c    0x4  Data  Lc  stm32f10x_rcc.o [1]
APBAHBPrescTable        0x20000400   0x10  Data  Lc  stm32f10x_rcc.o [1]
BusFault_Handler        0x08004adf    0x2  Code  Gb  stm32f10x_it.o [1]
CAN1_RX1_IRQHandler     0x08004ecb         Code  Wk  startup_stm32f10x_hd.o [1]
CAN1_SCE_IRQHandler     0x08004ecf         Code  Wk  startup_stm32f10x_hd.o [1]
CSTACK$$Base            0x20000000          --   Gb  - Linker created -
CSTACK$$Limit           0x20000400          --   Gb  - Linker created -
ConfigMsg               0x20000830   0x24  Data  Gb  device.o [1]
DHCP_REAL_SIP           0x20000878    0x4  Data  Gb  dhcp.o [1]
DHCP_SIP                0x20000874    0x4  Data  Gb  dhcp.o [1]
DHCP_XID                0x20000424    0x4  Data  Gb  dhcp.o [1]
DHCP_timeout            0x2000089a    0x1  Data  Gb  dhcp.o [1]
DHCP_timer              0x2000089b    0x1  Data  Gb  dhcp.o [1]
DMA1_Channel1_IRQHandler
                        0x08004ea3         Code  Wk  startup_stm32f10x_hd.o [1]
DMA1_Channel2_IRQHandler
                        0x08004ea7         Code  Wk  startup_stm32f10x_hd.o [1]
DMA1_Channel3_IRQHandler
                        0x08004eab         Code  Wk  startup_stm32f10x_hd.o [1]
DMA1_Channel4_IRQHandler
                        0x08004eaf         Code  Wk  startup_stm32f10x_hd.o [1]
DMA1_Channel5_IRQHandler
                        0x08004eb3         Code  Wk  startup_stm32f10x_hd.o [1]
DMA1_Channel6_IRQHandler
                        0x08004eb7         Code  Wk  startup_stm32f10x_hd.o [1]
DMA1_Channel7_IRQHandler
                        0x08004ebb         Code  Wk  startup_stm32f10x_hd.o [1]
DMA2_Channel1_IRQHandler
                        0x08004f57         Code  Wk  startup_stm32f10x_hd.o [1]
DMA2_Channel2_IRQHandler
                        0x08004f5b         Code  Wk  startup_stm32f10x_hd.o [1]
DMA2_Channel3_IRQHandler
                        0x08004f5f         Code  Wk  startup_stm32f10x_hd.o [1]
DMA2_Channel4_5_IRQHandler
                        0x08004f63         Code  Wk  startup_stm32f10x_hd.o [1]
DebugMon_Handler        0x08004ae5    0x2  Code  Gb  stm32f10x_it.o [1]
Delay_ms                0x08003d83   0x34  Code  Gb  util.o [1]
Delay_us                0x08003db7   0x34  Code  Gb  util.o [1]
EXTERN_DHCPBUF          0x20000430  0x400  Data  Gb  dhcp.o [1]
EXTI0_IRQHandler        0x08004e8f         Code  Wk  startup_stm32f10x_hd.o [1]
EXTI15_10_IRQHandler    0x08004f17         Code  Wk  startup_stm32f10x_hd.o [1]
EXTI1_IRQHandler        0x08004e93         Code  Wk  startup_stm32f10x_hd.o [1]
EXTI2_IRQHandler        0x08004e97         Code  Wk  startup_stm32f10x_hd.o [1]
EXTI3_IRQHandler        0x08004e9b         Code  Wk  startup_stm32f10x_hd.o [1]
EXTI4_IRQHandler        0x08004e9f         Code  Wk  startup_stm32f10x_hd.o [1]
EXTI9_5_IRQHandler      0x08004ed3         Code  Wk  startup_stm32f10x_hd.o [1]
FLASH_IRQHandler        0x08004e87         Code  Wk  startup_stm32f10x_hd.o [1]
FLASH_PrefetchBufferCmd
                        0x0800450f   0x1c  Code  Gb  stm32f10x_flash.o [1]
FLASH_SetLatency        0x080044f5   0x1a  Code  Gb  stm32f10x_flash.o [1]
FSMC_IRQHandler         0x08004f37         Code  Wk  startup_stm32f10x_hd.o [1]
GET_DNS_IP              0x2000041c    0x4  Data  Gb  dhcp.o [1]
GET_GW_IP               0x20000418    0x4  Data  Gb  dhcp.o [1]
GET_SIP                 0x20000420    0x4  Data  Gb  dhcp.o [1]
GET_SN_MASK             0x20000414    0x4  Data  Gb  dhcp.o [1]
GPIO_Configuration      0x0800309d   0xf2  Code  Gb  mcu_init.o [1]
GPIO_Init               0x08003741  0x150  Code  Gb  stm32f10x_gpio.o [1]
GPIO_ResetBits          0x08003897    0x6  Code  Gb  stm32f10x_gpio.o [1]
GPIO_SetBits            0x08003891    0x6  Code  Gb  stm32f10x_gpio.o [1]
HardFault_Handler       0x08004adb    0x2  Code  Gb  stm32f10x_it.o [1]
I2C1_ER_IRQHandler      0x08004ef7         Code  Wk  startup_stm32f10x_hd.o [1]
I2C1_EV_IRQHandler      0x08004ef3         Code  Wk  startup_stm32f10x_hd.o [1]
I2C2_ER_IRQHandler      0x08004eff         Code  Wk  startup_stm32f10x_hd.o [1]
I2C2_EV_IRQHandler      0x08004efb         Code  Wk  startup_stm32f10x_hd.o [1]
IINCHIP_CSoff           0x08002701    0xa  Code  Gb  w5500.o [1]
IINCHIP_CSon            0x0800270b    0xa  Code  Gb  w5500.o [1]
IINCHIP_READ            0x0800275b   0x3a  Code  Gb  w5500.o [1]
IINCHIP_SpiSendData     0x08002715    0xe  Code  Gb  w5500.o [1]
IINCHIP_WRITE           0x08002723   0x38  Code  Gb  w5500.o [1]
MemManage_Handler       0x08004add    0x2  Code  Gb  stm32f10x_it.o [1]
NMI_Handler             0x08004ad9    0x2  Code  Gb  stm32f10x_it.o [1]
NVIC_Configuration      0x08003221   0x70  Code  Gb  mcu_init.o [1]
NVIC_Init               0x080040cb   0x6e  Code  Gb  misc.o [1]
NVIC_PriorityGroupConfig
                        0x080040c1    0xa  Code  Gb  misc.o [1]
NVIC_SetVectorTable     0x08004139    0xc  Code  Gb  misc.o [1]
OLD_SIP                 0x2000087c    0x4  Data  Gb  dhcp.o [1]
PVD_IRQHandler          0x08004e7b         Code  Wk  startup_stm32f10x_hd.o [1]
PendSV_Handler          0x08004ae7    0x2  Code  Gb  stm32f10x_it.o [1]
RCC_ADCCLKConfig        0x08002c91   0x16  Code  Gb  stm32f10x_rcc.o [1]
RCC_APB1PeriphClockCmd  0x08002da9   0x1e  Code  Gb  stm32f10x_rcc.o [1]
RCC_APB2PeriphClockCmd  0x08002d8b   0x1e  Code  Gb  stm32f10x_rcc.o [1]
RCC_Configuration       0x0800318f   0x80  Code  Gb  mcu_init.o [1]
RCC_DeInit              0x08002b15   0x5c  Code  Gb  stm32f10x_rcc.o [1]
RCC_GetClocksFreq       0x08002ca7   0xe4  Code  Gb  stm32f10x_rcc.o [1]
RCC_GetFlagStatus       0x08002dc7   0x56  Code  Gb  stm32f10x_rcc.o [1]
RCC_GetSYSCLKSource     0x08002c43    0xa  Code  Gb  stm32f10x_rcc.o [1]
RCC_HCLKConfig          0x08002c4d   0x16  Code  Gb  stm32f10x_rcc.o [1]
RCC_HSEConfig           0x08002b71   0x4e  Code  Gb  stm32f10x_rcc.o [1]
RCC_IRQHandler          0x08004e8b         Code  Wk  startup_stm32f10x_hd.o [1]
RCC_PCLK1Config         0x08002c63   0x16  Code  Gb  stm32f10x_rcc.o [1]
RCC_PCLK2Config         0x08002c79   0x18  Code  Gb  stm32f10x_rcc.o [1]
RCC_PLLCmd              0x08002c21    0xa  Code  Gb  stm32f10x_rcc.o [1]
RCC_PLLConfig           0x08002c03   0x1e  Code  Gb  stm32f10x_rcc.o [1]
RCC_SYSCLKConfig        0x08002c2b   0x18  Code  Gb  stm32f10x_rcc.o [1]
RCC_WaitForHSEStartUp   0x08002bbf   0x44  Code  Gb  stm32f10x_rcc.o [1]
RSIZE                   0x20000864   0x10  Data  Lc  w5500.o [1]
RTCAlarm_IRQHandler     0x08004f1b         Code  Wk  startup_stm32f10x_hd.o [1]
RTC_IRQHandler          0x08004e83         Code  Wk  startup_stm32f10x_hd.o [1]
Region$$Table$$Base     0x080048d0          --   Gb  - Linker created -
Region$$Table$$Limit    0x080048f4          --   Gb  - Linker created -
Reset_Handler           0x08004dd9         Code  Wk  startup_stm32f10x_hd.o [1]
Reset_W5500             0x080039f5   0x26  Code  Gb  device.o [1]
SDIO_IRQHandler         0x08004f3b         Code  Wk  startup_stm32f10x_hd.o [1]
SPI1_IRQHandler         0x08004f03         Code  Wk  startup_stm32f10x_hd.o [1]
SPI2_IRQHandler         0x08004f07         Code  Wk  startup_stm32f10x_hd.o [1]
SPI2_SendByte           0x08004087   0x32  Code  Gb  SPI2.o [1]
SPI3_IRQHandler         0x08004f43         Code  Wk  startup_stm32f10x_hd.o [1]
SPI_Cmd                 0x080041a1   0x1a  Code  Gb  stm32f10x_spi.o [1]
SPI_I2S_GetFlagStatus   0x080041c3   0x1a  Code  Gb  stm32f10x_spi.o [1]
SPI_I2S_ReceiveData     0x080041bf    0x4  Code  Gb  stm32f10x_spi.o [1]
SPI_I2S_SendData        0x080041bb    0x4  Code  Gb  stm32f10x_spi.o [1]
SPI_Init                0x08004161   0x40  Code  Gb  stm32f10x_spi.o [1]
SRC_MAC_ADDR            0x20000410    0x4  Data  Gb  dhcp.o [1]
SSIZE                   0x20000854   0x10  Data  Lc  w5500.o [1]
SVC_Handler             0x08004ae3    0x2  Code  Gb  stm32f10x_it.o [1]
SetSysClock             0x080038ef    0x8  Code  Lc  system_stm32f10x.o [1]
SetSysClockTo72         0x080038f7   0xe0  Code  Lc  system_stm32f10x.o [1]
SysTick_Handler         0x08004ae9    0x2  Code  Gb  stm32f10x_it.o [1]
SystemInit              0x0800389d   0x52  Code  Gb  system_stm32f10x.o [1]
Systick_Init            0x08003d5d   0x26  Code  Gb  util.o [1]
TAMPER_IRQHandler       0x08004e7f         Code  Wk  startup_stm32f10x_hd.o [1]
TIM1_BRK_IRQHandler     0x08004ed7         Code  Wk  startup_stm32f10x_hd.o [1]
TIM1_CC_IRQHandler      0x08004ee3         Code  Wk  startup_stm32f10x_hd.o [1]
TIM1_TRG_COM_IRQHandler
                        0x08004edf         Code  Wk  startup_stm32f10x_hd.o [1]
TIM1_UP_IRQHandler      0x08004edb         Code  Wk  startup_stm32f10x_hd.o [1]
TIM2_IRQHandler         0x08004aeb    0x2  Code  Gb  stm32f10x_it.o [1]
TIM3_IRQHandler         0x08004aed    0x2  Code  Gb  stm32f10x_it.o [1]
TIM4_IRQHandler         0x08004eef         Code  Wk  startup_stm32f10x_hd.o [1]
TIM5_IRQHandler         0x08004f3f         Code  Wk  startup_stm32f10x_hd.o [1]
TIM6_IRQHandler         0x08004f4f         Code  Wk  startup_stm32f10x_hd.o [1]
TIM7_IRQHandler         0x08004f53         Code  Wk  startup_stm32f10x_hd.o [1]
TIM8_BRK_IRQHandler     0x08004f23         Code  Wk  startup_stm32f10x_hd.o [1]
TIM8_CC_IRQHandler      0x08004f2f         Code  Wk  startup_stm32f10x_hd.o [1]
TIM8_TRG_COM_IRQHandler
                        0x08004f2b         Code  Wk  startup_stm32f10x_hd.o [1]
TIM8_UP_IRQHandler      0x08004f27         Code  Wk  startup_stm32f10x_hd.o [1]
UART4_IRQHandler        0x08004f47         Code  Wk  startup_stm32f10x_hd.o [1]
UART5_IRQHandler        0x08004f4b         Code  Wk  startup_stm32f10x_hd.o [1]
USART1_IRQHandler       0x08004aef    0x2  Code  Gb  stm32f10x_it.o [1]
USART1_Init             0x08003a1b   0x48  Code  Gb  device.o [1]
USART2_IRQHandler       0x08004af1    0x2  Code  Gb  stm32f10x_it.o [1]
USART3_IRQHandler       0x08004f13         Code  Wk  startup_stm32f10x_hd.o [1]
USART_Cmd               0x0800351d   0x1a  Code  Gb  stm32f10x_usart.o [1]
USART_GetFlagStatus     0x0800359d   0x22  Code  Gb  stm32f10x_usart.o [1]
USART_ITConfig          0x08003537   0x5e  Code  Gb  stm32f10x_usart.o [1]
USART_Init              0x08003435   0xe2  Code  Gb  stm32f10x_usart.o [1]
USART_SendData          0x08003595    0x8  Code  Gb  stm32f10x_usart.o [1]
USBWakeUp_IRQHandler    0x08004f1f         Code  Wk  startup_stm32f10x_hd.o [1]
USB_HP_CAN1_TX_IRQHandler
                        0x08004ec3         Code  Wk  startup_stm32f10x_hd.o [1]
USB_LP_CAN1_RX0_IRQHandler
                        0x08004ec7         Code  Wk  startup_stm32f10x_hd.o [1]
UsageFault_Handler      0x08004ae1    0x2  Code  Gb  stm32f10x_it.o [1]
WIZ_CS                  0x0800405f   0x28  Code  Gb  SPI2.o [1]
WIZ_SPI_Init            0x0800400d   0x52  Code  Gb  SPI2.o [1]
WWDG_IRQHandler         0x08004e77         Code  Wk  startup_stm32f10x_hd.o [1]
_GenldDefault           0x08001fb9  0x24e  Code  Lc  xprintffull.o [3]
_LdtobDefault           0x08001ba5  0x40e  Code  Lc  xprintffull.o [3]
_LitobDefault           0x08001a97  0x10e  Code  Lc  xprintffull.o [3]
_Printf                 0x08001591  0x506  Code  Gb  xprintffull.o [3]
_Prout                  0x08004c87   0x16  Code  Gb  xprout.o [3]
_PutcharsDefault        0x08002221   0x32  Code  Lc  xprintffull.o [3]
_SProut                 0x08004e03    0xa  Code  Gb  xsprout.o [3]
__aeabi_cdcmple         0x080045fd         Code  Gb  DblCmpLe.o [4]
__aeabi_cdrcmple        0x0800462d         Code  Gb  DblCmpGe.o [4]
__aeabi_d2iz            0x080043dd         Code  Gb  DblToI32.o [4]
__aeabi_d2uiz           0x08004409         Code  Gb  DblToI32.o [4]
__aeabi_dadd            0x08003e61         Code  Gb  DblAdd.o [4]
__aeabi_ddiv            0x08002e55         Code  Gb  DblDiv.o [4]
__aeabi_dmul            0x08003291         Code  Gb  DblMul.o [4]
__aeabi_dsub            0x080035c1         Code  Gb  DblSub.o [4]
__aeabi_i2d             0x0800465d         Code  Gb  I32ToDbl.o [4]
__aeabi_ldiv0           0x08004e51         Code  Gb  I64DivZer.o [4]
__aeabi_ldivmod         0x08003b25         Code  Gb  I64DivMod.o [4]
__aeabi_memcpy          0x080041dd         Code  Gb  ABImemcpy.o [4]
__aeabi_memcpy4         0x080041f7         Code  Gb  ABImemcpy.o [4]
__aeabi_memcpy8         0x080041f7         Code  Gb  ABImemcpy.o [4]
__aeabi_memset          0x080042b9         Code  Gb  ABImemset.o [4]
__aeabi_ui2d            0x08004671         Code  Gb  I32ToDbl.o [4]
__aeabi_uldivmod        0x08003b39         Code  Gb  I64DivMod.o [4]
__exit                  0x08004d65   0x14  Code  Gb  exit.o [5]
__iar_Dnorm             0x08003f47   0xc6  Code  Gb  xdnorm.o [3]
__iar_Dscale            0x08003c55  0x108  Code  Gb  xdscale.o [3]
__iar_Memchr            0x08004385         Code  Gb  memchr.o [4]
__iar_Memset            0x080042b9         Code  Gb  ABImemset.o [4]
__iar_Memset_word       0x080042c1         Code  Gb  ABImemset.o [4]
__iar_Strchr            0x08004c45         Code  Gb  strchr.o [4]
__iar_copy_init2        0x080048ad   0x24  Code  Gb  copy_init2.o [4]
__iar_d2uiz             0x08004413         Code  Gb  DblToI32.o [4]
__iar_dadd              0x08003e73         Code  Gb  DblAdd.o [4]
__iar_data_init2        0x080049f5   0x20  Code  Gb  data_init2.o [4]
__iar_dsub              0x080035d3         Code  Gb  DblSub.o [4]
__iar_dsubStart         0x080035e5         Code  Gb  DblSub.o [4]
__iar_program_start     0x08004c2d         Code  Gb  cmain.o [4]
__iar_sh_stdout_close   0x08004abd   0x16  Code  Gb  iarwstd.o [5]
__iar_sh_stdout_handle  0x20000890    0x4  Data  Lc  iarwstd.o [5]
__iar_ui2d              0x08004673         Code  Gb  I32ToDbl.o [4]
__iar_zero_init2        0x08004af3   0x1a  Code  Gb  zero_init2.o [4]
__low_level_init        0x08004f67    0x4  Code  Gb  low_level_init.o [3]
__vector_table          0x08000000         Data  Gb  startup_stm32f10x_hd.o [1]
_exit                   0x08004df9         Code  Gb  cexit.o [4]
_main                   0x08004c3f         Code  Gb  cmain.o [4]
at24c16_init            0x080044b9   0x38  Code  Gb  at24c16.o [1]
check_DHCP_Timeout      0x080012ed   0x84  Code  Gb  dhcp.o [1]
check_DHCP_state        0x080010d9  0x210  Code  Gb  dhcp.o [1]
check_leasedIP          0x08001371   0x54  Code  Gb  dhcp.o [1]
close                   0x0800233f   0x32  Code  Gb  socket.o [1]
dhcp_lease_time         0x20000880    0x4  Data  Gb  dhcp.o [1]
dhcp_retry_count        0x20000899    0x1  Data  Gb  dhcp.o [1]
dhcp_state              0x20000898    0x1  Data  Gb  dhcp.o [1]
dhcp_tick_cnt           0x2000088c    0x4  Data  Gb  dhcp.o [1]
dhcp_time               0x20000884    0x4  Data  Gb  dhcp.o [1]
div                     0x08004de9    0xe  Code  Gb  div.o [3]
exit                    0x08004e35    0x6  Code  Gb  exit.o [3]
fac_ms                  0x20000896    0x2  Data  Lc  util.o [1]
fac_us                  0x2000089c    0x1  Data  Lc  util.o [1]
getIINCHIP_TxMAX        0x080026f5    0xc  Code  Gb  w5500.o [1]
getSn_RX_RSR            0x08002a07   0x6c  Code  Gb  w5500.o [1]
getSn_SR                0x080029f5   0x12  Code  Gb  w5500.o [1]
htonl                   0x08004797    0xc  Code  Gb  sockutil.o [1]
htons                   0x08004789    0xe  Code  Gb  sockutil.o [1]
iinchip_init            0x08002853    0xa  Code  Gb  w5500.o [1]
init_dhcp_client        0x080013c5   0xac  Code  Gb  dhcp.o [1]
local_port              0x20000894    0x2  Data  Lc  socket.o [1]
main                    0x0800424d   0x6c  Code  Gb  main.o [1]
memchr                  0x08004385         Code  Gb  memchr.o [4]
memcmp                  0x08004321         Code  Gb  memcmp.o [4]
memcpy                  0x08004c5b   0x16  Code  Gb  device.o [1]
memset                  0x08004c71   0x16  Code  Gb  dhcp.o [1]
next_dhcp_time          0x20000888    0x4  Data  Gb  dhcp.o [1]
ntohl                   0x080047a3    0xc  Code  Gb  sockutil.o [1]
pRIPMSG                 0x20000428    0x4  Data  Gb  dhcp.o [1]
parseDHCPMSG            0x08000c61  0x46c  Code  Gb  dhcp.o [1]
printf                  0x080049d5   0x20  Code  Gb  printf.o [3]
putchar                 0x08003deb   0x2a  Code  Gb  util.o [1]
recvfrom                0x080024a5  0x244  Code  Gb  socket.o [1]
reset_DHCP_time         0x08000131   0x28  Code  Gb  dhcp.o [1]
send_DHCP_DISCOVER      0x08000159  0x354  Code  Gb  dhcp.o [1]
send_DHCP_RELEASE_DECLINE
                        0x08000919  0x320  Code  Gb  dhcp.o [1]
send_DHCP_REQUEST       0x080004ad  0x46c  Code  Gb  dhcp.o [1]
send_data_processing    0x08002a73   0x90  Code  Gb  w5500.o [1]
sendto                  0x08002371  0x134  Code  Gb  socket.o [1]
setGAR                  0x0800299d   0x12  Code  Gb  w5500.o [1]
setMR                   0x080029e5   0x10  Code  Gb  w5500.o [1]
setSHAR                 0x080029c1   0x12  Code  Gb  w5500.o [1]
setSIPR                 0x080029d3   0x12  Code  Gb  w5500.o [1]
setSUBR                 0x080029af   0x12  Code  Gb  w5500.o [1]
set_default             0x08003a63   0x8c  Code  Gb  device.o [1]
socket                  0x08002255   0xea  Code  Gb  socket.o [1]
sprintf                 0x080045cd   0x30  Code  Gb  sprintf.o [3]
strchr                  0x08004c45         Code  Gb  strchr.o [4]
strcpy                  0x08004435         Code  Gb  strcpy.o [4]
strlen                  0x08004531         Code  Gb  strlen.o [4]
swapl                   0x08003e29   0x20  Code  Gb  util.o [1]
swaps                   0x08003e15   0x14  Code  Gb  util.o [1]
sysinit                 0x0800285d  0x140  Code  Gb  w5500.o [1]
wiz_read_buf            0x080027f5   0x5e  Code  Gb  w5500.o [1]
wiz_write_buf           0x08002795   0x60  Code  Gb  w5500.o [1]


[1] = E:\WIZnet 产品文档\W5500\W5500\Application Reference\DHCP test\DHCP test\Debug\Obj
[2] = command line
[3] = dl7M_tl_in.a
[4] = rt7M_tl.a
[5] = shb_l.a

  18 582 bytes of readonly  code memory
   1 798 bytes of readonly  data memory
   2 205 bytes of readwrite data memory

Errors: none
Warnings: none
